:020000000528D1
:10000800212883160030850001308600C030810029
:1000180006309F00831200309200D8200821B201D8
:10002800E1010D30C30064307B2164307B218B10EB
:100038000B168B1706308A0047288B138B100B1270
:10004800831340212A21B500B03E03182F28B2128D
:100058003508A03E3128B216203EA0008313562151
:10006800B500B21A83172008840035080D3A031921
:10007800452807308A003508E03ED7208000A00ACE
:10008800322883131928E5203230FE2025212C3010
:10009800A20000005D30FD202521A20B4D28A030D4
:1000A800A3008313BC30A200A501AB015830FE2089
:1000B8000230FE2025210530FE2025085F3A031D69
:1000C8006B280000AB012030A300831770280000C4
:1000D8000000000000007028230884002B08063C5C
:1000E800031C782898207B2800004830FC20251C19
:1000F800AB0A2B080C3A031D8528AB011430A30763
:1001080088280000000088280000A50AA20B5C28A7
:100118000730FD201730A20025215F30FE20A20BFA
:100128009028252102214728D42093000000D420BC
:1001380093000000D42093000000D4209300000016
:10014800D42093000000D42093000000D420930012
:100158000000D42093000000D42093000000D42095
:1001680093000000D42093000000D42093000000E6
:10017800D42093000000D42093000000D4209300E2
:100188000000D42093000000D42093000000D42065
:1001980093000000D42093000000D42093000800AE
:1001A8000008840A2B07820083168030940083128B
:1001B8002030940008008316141CE0288312930052
:1001C80008000630B50025212A30FE20B50BE728A7
:1001D8000730B50020212A30FE20B50BEE28063066
:1001E800B500202125212A30FE20B50BF62808006D
:1001F80000000000B100B10BFF280800000000005B
:100208005F300629FE2008008313A03084002030C8
:100218001421831720308400203014218313080010
:10022800B5005030AE0007308A003508D72080006E
:10023800840AAE0B1929080086150430FE208611A1
:10024800080086110430FE2086150800C0015621DA
:10025800B5003030B502031C3E290A3035020318B8
:100268003E290310C00D4008C00DC00DC007350859
:10027800C0072B2940080800E10160216400B5008F
:100288000B3A0319052861081C3A0319E1034330A6
:100298006107E10A8400350880000D3A031D4129F1
:1002A800E101080043306107E10A840000080D3AC3
:1002B8000319E10300080800AE01AE15B501061CDC
:1002C80063297621061C602974210310061C031477
:1002D800B50C00000000AE0B682974213508080031
:1002E800A43077295230EA00EA0B78290800A800E0
:1002F8008A21A80B7C29080001308B2902308B2920
:1003080005308B290A308B2932308B296430A700BD
:100318000000000000000E30A600A60B9129A70BD4
:040328008C29080014
:100C0000FC3482348234FC3482348234FC348034C8
:100C1000803480347C348234803480348034823434
:100C20007C348234803480348E3482347C34FE349C
:100C300080348034FE3480348034FE348034803418
:100C40008034803480348034FE34103410341034D6
:100C50001034103410341034383444348234823434
:100C6000FE34823482348234FE34823482348234DC
:100C70008234823482347C34823480347C34023452
:100C800082347C34823402343C3440348034FE3448
:100C90000234043408341034303410341034103436
:100CA000103410347C34823402340C3402348234F4
:100CB0007C34823482347C34823482347E34023414
:100CC00002347C34FC348234823482348234823480
:100CD000FC3482348234FC348234823482342834CA
:100CE000023402347C34823482348234FE3402345E
:100CF000023402340234023482347C347C34823450
:100D00008A349234A23482347C347C34803480340B
:100D1000FC34823482347C34823484348834E03449
:100D20008834843482348234C634AA34923482348F
:100D300082348234823444342834103428344434A5
:100D400082348234C234A23492348A348634823477
:100D5000823482349234AA34C6348234FE34043469
:100D60000834103420344034FE3480348034FC3471
:100D7000023402347C347C348234823482348234CF
:100D800082347C347C348234823482348A348634B3
:100D90007C3482340234043408340034083400349F
:100DA0000034003400340034003400340834083493
:100DB000103400340034003400340034003406347D
:100DC0000634003400347C3400347C340034003485
:100DD00000347C34003400340034023404340834E9
:100DE000103420344034103410341034FE341034B5
:100DF000103410349234543438345434923410341F
:100E0000CF34CF34CF34CF34CF34CF34CF34CF34CA
:100E1000CF34CF34F934F334D234E634DA34EC342A
:100E20007E344C34413452347334B43485344734D2
:100E300058345B34CF34CF34CF34E134CF34C8347A
:100E4000CF342C3400340A34623417341A3410345A
:100E50003134253477348C341E349334A134BB348C
:100E60000334C23468343B34243435349734A734E3
:100E70009A346C34AE34CF34CF34CF34CF34CF3413
:100E8000CF342C3400340A34623417341A3410341A
:100E90003134253477348C341E349334A134BB344C
:100EA0000334C23468343B34243435349734A734A3
:100EB0009A346C34AE34CF34CF34CF34CF34CF34D3
:02400E00222F5F
:00000001FF
